:1000000012C02CC02BC02AC08BC028C027C026C05D
:1000100025C0C8C023C022C021C020C01FC01EC030
:100020001DC01CC01BC011241FBECFE5D4E0DEBF25
:10003000CDBF10E0A0E6B0E0E2E7F7E002C0059037
:100040000D92A43BB107D9F710E0A4EBB0E001C0DA
:100050001D92A43CB107E1F794D089C3D1CFC29AD5
:1000600000000000C298089511BAC09AC19801C05A
:10007000F6DF82B38035E0F78FEF81BB08951F93E1
:10008000182FF2DF12BB88B38C7F88BBE8DF12BA6F
:100090001F9108951F9387B3876087BB86EA9EE010
:1000A0000197F1F781E0EBDF84EF91E00197F1F741
:1000B00088E3E5DF10E1812F8A95F1F78CE0DFDF3F
:1000C0001A95F1F71F9108951F93182FCDDF12BBDA
:1000D000C098C19AC4DF12BA1F910895CF93DF93DD
:1000E000EC0102C02196F0DF88818823D9F7DF91E7
:1000F000CF9108958158ECEAF0E0E60FF11D908170
:10010000890FBDDF089588E082BD83B7846083BF17
:1001100085B5856085BD89B7816489BF7894089568
:100120001F920F920FB60F9211248F938091B500FA
:10013000813009F58091B40081508093B4008F3FE5
:1001400041F48BE38093B4008091B200815080939E
:10015000B2008091B200882329F48091B4008823F2
:1001600051F406C08F3F39F48091B400873318F002
:1001700083E08093B6008F910F900FBE0F901F9079
:100180001895C1DF87DF87B3886187BB88B3877E17
:1001900088BBA59AAD9884B3817E84BB85B38E61FC
:1001A00085BBFFCF1F920F920FB60F9211241F93A2
:1001B0002F933F934F935F936F937F938F939F936F
:1001C000AF93BF93EF93FF93AD98999B03C084E0E7
:1001D0008093B6008091B40090E06CEB70E04AE050
:1001E00050E082D28091B20090E060EC70E04AE092
:1001F00050E07AD28091B600882309F096C081E061
:1002000061E078DF80E690E069DF82E062E072DF43
:100210008091B2008A3018F489E690E05FDF80ECCC
:1002200090E05CDF8BE690E059DF8091B4008A308B
:1002300018F48DE690E052DF8CEB90E04FDF88B34E
:10024000877E88BB9C9B04C09A9B02C09B9905C07B
:100250008091B7008F5F8093B7009C9B0BC09A9BE7
:1002600009C09B9B07C01092B7001092BB008AE0A8
:100270008093B1008091BB00863030F082E08093A3
:10028000B10086E08093BB009091B7008091B100EF
:10029000981708F44AC09C9908C0AD9A81E08093F1
:1002A000B9008093B6001092B7009A9917C0AD9A22
:1002B0009091B400965F9093B4008091BB008F5FE3
:1002C0008093BB001092B7009C539F3038F480910C
:1002D000B2008F5F8093B2009093B4009B9925C0C9
:1002E000AD9A2091B400922F9A509093B4008091CF
:1002F000BB008F5F8093BB001092B700963F40F029
:100300008091B20081508093B2002E5C2093B400A3
:100310008091B200882349F48091B400882329F4A5
:100320001092B2008AE08093B4008091B6008130D0
:1003300009F095C08093B50061E0DCDE8FE690E0C7
:10034000CDDE82E062E0D6DE8091B2008A3018F421
:1003500089E690E0C3DE80EC90E0C0DE8BE690E0C2
:10036000BDDE8091B4008A3018F48DE690E0B6DEF0
:100370008CEB90E0B3DE88B3886188BB9C9B04C0A3
:100380009A9B02C09B9905C08091B7008F5F8093B4
:10039000B7009C9B0BC09A9B09C09B9B07C0109207
:1003A000B7001092BB008AE08093B1008091BB003F
:1003B000863030F082E08093B10086E08093BB000D
:1003C0009091B7008091B100981708F448C09C99AB
:1003D00006C0AD9A82E08093B6001092B7009A9959
:1003E00017C0AD9A9091B400965F9093B40080913D
:1003F000BB008F5F8093BB001092B7009C539F306F
:1004000038F48091B2008F5F8093B2009093B40073
:100410009B9925C0AD9A8091BB008F5F8093BB00F4
:100420001092B7002091B200222371F09091B40095
:10043000892F8A508093B400863F30F0215020935A
:10044000B2009E5C9093B4008091B200882339F48E
:100450008091B4008A3018F08A508093B400809163
:10046000B600823009F096C01092B50081E061E0DC
:1004700041DE88E790E032DE82E062E03BDE8091A0
:10048000B2008A3018F489E690E028DE80EC90E033
:1004900025DE8BE690E022DE8091B4008A3018F4ED
:1004A0008DE690E01BDE8CEB90E018DE88B3877E53
:1004B00088BB9C9B04C09A9B02C09B9905C08091FD
:1004C000B7008F5F8093B7009C9B0BC09A9B09C0BD
:1004D0009B9B07C01092B7001092BB008AE08093EC
:1004E000B1008091BB00863030F082E08093B10093
:1004F00086E08093BB009091B7008091B10098177F
:1005000008F448C09C9906C0AD9A81E08093B6007B
:100510001092B7009A9917C0AD9A9091B400965F67
:100520009093B4008091BB008F5F8093BB001092CA
:10053000B7009C539F3038F48091B2008F5F809356
:10054000B2009093B4009B9925C0AD9A8091BB00F6
:100550008F5F8093BB001092B7002091B2002223DE
:1005600071F09091B400892F8A508093B400863F37
:1005700030F021502093B2009E5C9093B4008091A3
:10058000B200882339F48091B4008A3018F08A5080
:100590008093B4008091B600833009F044C010927B
:1005A000B50081E08093BA0061E0A4DD81E890E0CD
:1005B00095DD81E062E09EDD8AE890E08FDD80914C
:1005C000B800882321F0823011F0843009F4AD9A0C
:1005D0008F5F8093B80088B3877E88BB9C9905C0E5
:1005E0008091B7008F5F8093B7009C9B02C01092F0
:1005F000B7009091B7008091B1009817A0F0AD9A24
:1006000081E062E077DD83E990E068DD1092B6007A
:100610001092B90081E08093B2001092B80010925D
:10062000B7001092BA008091B600843009F04AC039
:100630001092B50081E061E05DDD8CE990E04EDD77
:1006400081E062E057DD85EA90E048DD88B3877E8F
:1006500088BB99990CC08091B900882341F410920D
:10066000B60081E062E046DD83E990E037DD9999EC
:1006700011C08091B900813069F48091BA0088235B
:1006800049F482E08093B60081E062E033DD83E9E3
:1006900090E024DD999916C01091BA00113091F4C0
:1006A0001092B60081E062E025DD83E990E016DD7E
:1006B0001092B9001093B2001092B8001092B700D7
:1006C0001092BA00FF91EF91BF91AF919F918F91DE
:1006D0007F916F915F914F913F912F911F910F905B
:1006E0000FBE0F901F901895FB019F01E8944230B8
:1006F000BCF04532ACF44A3029F497FB1EF49095D7
:1007000081959F4F642F77271ED0805D8A330CF030
:10071000895D8193CB010097A9F716F45DE25193AF
:100720001082C90100C0DC01FC01672F71917723A1
:10073000E1F7329704C07C916D9370836291AE179C
:10074000BF07C8F30895AA1BBB1B51E107C0AA1F2E
:10075000BB1FA617B70710F0A61BB70B881F991F62
:100760005A95A9F780959095BC01CD010895F8940C
:02077000FFCFB9
:100772005345542054494D450020003A003000456D
:1007820058504F53494E470020504155534544203D
:10079200004558504F5355524500434F4D504C451C
:1007A20054450020202020202020200020494E53A4
:1007B200455254200020424F41524421000040142F
:0407C200540A0100D4
:00000001FF
